:100000008E28A00062200C080D0403198928832083
:1000100084132008800664000D280E288C0A03191A
:100020008D0F0B288006892823088C0021088D005D
:1000300001308E008F0164003C20031C2F288E0BA2
:100040001B28FF308F0703181B288C07031C8D0704
:10005000031C892832308E0000308F001B28472077
:1000600008308F0048203C208E0C36288F0B322819
:10007000482003140E080800220884002008841772
:100080008004841300051F192006FF3E08001F1777
:100090001F0D06398C0056208D008C0A56201F1F1C
:1000A00067281F138C0002307E20672800308A00EA
:1000B0000C088207013475340334153400343C34A1
:1000C0000C34D934FF3A8417800589288D01E83E25
:1000D0008C008D09FC30031C70288C0703186D28D8
:1000E0008C0764008D0F6D280C1876288C1C7A28DC
:1000F00000007A28080003108D0C8C0CFF3E0318BA
:100100007B280C0889288C098D098C0A03198D0A13
:10011000080083130313831264000800831686010A
:10012000FF30850083120610831606108312861096
:100130008316861083120611831606118312861108
:1001400083168611831206128316061283128612F4
:1001500083168612831206138316061383128613E0
:1001600083168613831205168316051283127F30B9
:10017000A7006F30A8009030A9004130AA007F305E
:10018000AB007F30AC007F30AD007F30AE0001307F
:10019000A6000B30A4000530A2000130A0000430FE
:1001A0009F000730A300A1011420031C9229FF3CEB
:1001B000031DD4281420031C9229A40064002408E1
:1001C000013C031DEC282608A70264002830270202
:1001D0000318EC282830A70064002408023C031D03
:1001E000FA282608A7076400E7302702031CFA282C
:1001F000E630A70064002408033C031D0B292608F1
:10020000A802640028302802031808292830A80012
:100210002808FE3CA90064002408043C031D1C2996
:100220002608A8076400E7302802031C1929E630D5
:10023000A8002808FE3CA90064002408053C031D12
:100240002A292608AA076400E7302A02031C2A2963
:10025000E630AA0064002408063C031D382926085D
:10026000AA02640028302A02031838292830AA007C
:1002700064002408073C031D49292608AB026400DA
:1002800028302B02031846292830AB002B08FE3CEF
:10029000AC0064002408083C031D5A292608AB075B
:1002A0006400E7302B02031C5729E630AB002B0813
:1002B000FE3CAC0064002408093C031D68292608A4
:1002C000AD076400E7302D02031C6829E630AD005D
:1002D000640024080A3C031D76292608AD02640048
:1002E00028302D02031876292830AD006400240838
:1002F0000B3C031D84292608AE0264000A302E023E
:10030000031884290A30AE00640024080C3C031D45
:1003100092292608AE076400E7302E02031C9229BA
:10032000E630AE0027088C008D01063084000130D5
:10033000012028088C008D01063084000230012045
:1003400029088C008D0106308400043001202A0821
:100350008C008D0106308400083001202B088C00B1
:100360008D0106308400103001202C088C008D0196
:1003700006308400203001202D088C008D010630CD
:100380008400403001202E088C008D01063084004E
:0603900080300120CB28A3
:02400E00F53F7C
:00000001FF
